:0400000048EF3FF096
:107E900000014BEF3FF0000E956EFC0E946E936860
:107EA000000E836E82B657EF3FF059EF3FF060EF60
:107EB0003FF094947E0ECA6E2F0EBD6E3E0EBE6EC7
:107EC00082A865EF3FF067EF3FF06EEF3FF09494CC
:107ED0007E0ECA6E0F0EBD6E7D0EBE6E81BA73EF42
:107EE0003FF075EF3FF052EF3FF094947E0ECA6E74
:107EF0002F0EBD6EBB0EBE6E52EF3FF000EF00F0D6
:020000040020DA
:08000000FFFFFFFFFFFFFFFF00
:020000040030CA
:0E000000FF071F1FFF8285FF0FC00FE00F409C
:00000001FF
